:100000000C9463000C94CC070C94F9070C948B00AF
:100010000C948B000C948B000C948B000C948B0034
:100020000C948B000C948B000C948B000C948B0024
:100030000C948B000C948B000C948B000C948B0014
:100040000C9426080C948B000C94F3090C94450A2C
:100050000C948B000C948B000C948B000C948B00F4
:100060000C948B000C948B000000000024002700EF
:100070002A0000000000250028002B0000000000DE
:1000800023002600290004040404040404040202DA
:100090000202020203030303030301020408102007
:1000A0004080010204081020010204081020000012
:1000B0000007000201000003040600000000000029
:1000C0000000B400B60B11241FBECFEFD8E0DEBF96
:1000D000CDBF11E0A0E0B1E0E0E8FBE102C0059097
:1000E0000D92A83CB107D9F712E0A8ECB1E001C02D
:1000F0001D92AF39B107E1F710E0C6ECD0E004C0C3
:100100002297FE010E94BA0DC23CD107C9F70E9496
:100110000D0C0C94BE0D0C9400001092D70110929F
:10012000D6012091D8013091D9018091E0019091C0
:10013000E10128173907B9F021153105A1F03093F5
:10014000E1012093E0018091DA019091DB0190932D
:10015000E3018093E2011092D9011092D80110922C
:10016000DB011092DA01089588EC91E06AE049E041
:100170000E9487070895F8948091D6019091D70145
:10018000803191052CF46091E0017091E10105C08E
:1001900040976091E2017091E30102C07695679506
:1001A0008A95E2F7617084E00E944B098AE090E052
:1001B0000E94C7088091D6019091D7014097BCF565
:1001C00085E00E949F09892BC1F081E090E0A0E0CA
:1001D000B0E00090D60104C0880F991FAA1FBB1F72
:1001E0000A94D2F72091E0013091E101282B392BBC
:1001F0003093E1012093E00154C081E090E0A0E061
:10020000B0E00090D60104C0880F991FAA1FBB1F41
:100210000A94D2F7809590952091E0013091E10108
:10022000822393239093E1018093E0013AC085E01B
:100230000E949F092091D6013091D701892BC1F0EE
:100240002051304081E090E0A0E0B0E004C0880F91
:10025000991FAA1FBB1F2A95D2F72091E201309166
:10026000E301282B392B3093E3012093E20119C0DD
:100270002051304081E090E0A0E0B0E004C0880F61
:10028000991FAA1FBB1F2A95D2F7809590952091A0
:10029000E2013091E301822393239093E301809361
:1002A000E2018091D6019091D701019660E270E061
:1002B0000E94630D9093D7018093D601789408959E
:1002C0001F93CF93DF9388EC91E00E9488058823E9
:1002D00039F088EC91E00E943C07882309F0B1C016
:1002E00065E070E080E090E00E946E08B2C08DE7AB
:1002F00092E060E071E00E941A0D8DE792E060915B
:10030000C8014AE050E00E94080D8DE792E00E948B
:10031000480C8DE792E06BE071E00E941A0D10E04E
:100320001BC0C12FD0E0FE01E853FE4F8181803118
:1003300018F06AE171E002C06CE171E08DE792E0D3
:100340000E941A0DC853DE4F8DE792E0698140E1AB
:1003500050E00E94080D1F5F8091C801181708F334
:100360008DE792E00E94480C8DE792E06FE171E02A
:100370000E941A0D10E01BC0C12FD0E0FE01E8530F
:10038000FE4F8181803118F06AE171E002C06CE1BA
:1003900071E08DE792E00E941A0DC853DE4F8DE7A1
:1003A00092E0698142E050E00E94080D1F5F809159
:1003B000C801181708F38DE792E00E94480C80915D
:1003C000C9016091CA010E94300D90689093D901D3
:1003D0008093D8018091CB016091CC010E94300DB7
:1003E0009093DB018093DA018DE792E00E94B40BD9
:1003F000882379F18DE792E06EE271E00E941A0D98
:100400006091D8017091D9018DE792E042E050E00F
:100410000E94F70C8DE792E06AE171E00E941A0DEC
:100420006091DA017091DB018DE792E042E050E0EB
:100430000E94F70C8DE792E06EE371E00E941D0DC3
:1004400008C08DE792E00E94B40B882309F4B7CF6F
:100450004ECFDF91CF911F9108951F938DE792E0CA
:1004600040E051EE60E070E00E94800A0E949C0231
:1004700088EC91E00E9446078DE792E00E94B40B61
:10048000882341F18DE792E06FE371E00E941D0D3A
:1004900088EC91E06EE60E941203182F8DE792E03F
:1004A00067E571E00E941A0D8DE792E0612F40E14F
:1004B00050E00E94080D11501E3F30F08DE792E091
:1004C00064E771E00E941D0D8DE792E06EE371E03C
:1004D0000E941D0D82E062E00E940C0980E06BEB3F
:1004E00070E043E050E00E94A90783E062E00E94D0
:1004F0000C0981E06DE870E043E050E00E94A9073C
:1005000085E060E00E940C0984E061E00E940C0933
:1005100084E060E00E944B091F910895882319F43C
:100520008CB5806202C08CB58F7D8CBD08959CB562
:10053000937F982B9CBD08958AE061E00E944B094F
:100540008AE061E00E940C098CB580618CBD8CB59D
:1005500080648CBD8DE061E00E940C098BE061E05D
:100560000E940C090895CF92DF92FF920F931F9380
:10057000CF93DF936C01F42EE901442309F44AC0C0
:10058000162F1E771068FC01848560E00E944B09DD
:100590004F2D41501EBD0DB407FEFDCF8EB5FE019F
:1005A00050E061E070E027C05523E9F40023D9F062
:1005B000202F30E009C0CB01022E02C0880F991F06
:1005C0000A94E2F7382B2F5F2830A8F31EBD0DB434
:1005D00007FEFDCF8EB5932F909528819223382367
:1005E000932B988306C01EBD0DB407FEFDCF8EB5BC
:1005F00080835F5F31965417B8F21EBC0DB407FEBE
:10060000FDCF8EB5C40FD11D8883F601848561E0CE
:100610000E944B09DF91CF911F910F91FF90DF90C6
:10062000CF9008951F93CF93DF93EC01162F8C8505
:1006300060E00E944B091E7710681EBD0DB407FED6
:10064000FDCF8EB51EBC0DB407FEFDCF1EB58C854B
:1006500061E00E944B09812FDF91CF911F91089596
:10066000EF92FF920F931F93CF93DF93EC01162F1E
:10067000E42E022FF32E8C8560E00E944B091E773A
:100680001EBD0DB407FEFDCF8EB5802F9F2D9C01A2
:10069000F90190E008C080818EBD0DB407FEFDCF4A
:1006A0008EB59F5F31969E15B0F38C8561E00E94F8
:1006B0004B09DF91CF911F910F91FF90EF9008951B
:1006C0000F931F93CF93DF93EC01162F042F8C858C
:1006D00060E00E944B091E771EBD0DB407FEFDCFE2
:1006E0008EB50EBD0DB407FEFDCF8EB58C8561E0D5
:1006F0000E944B09DF91CF911F910F910895CF93E5
:10070000DF93EC0168E20E941203482F837083306C
:1007100029F04360CE0168E20E946003DF91CF912F
:100720000895CF93DF93EC0162E04FE00E946003F5
:1007300062E370E080E090E00E946E08CE0162E02B
:100740000E94120384FDFACFDF91CF910895EF92BA
:10075000FF920F931F938C01E62EF42E0E9412033A
:10076000F094F822C8016E2D4F2D0E9460031F9156
:100770000F91FF90EF900895EF92FF920F931F93C8
:100780008C01E62EF42E0E941203F82AC8016E2D69
:100790004F2D0E9460031F910F91FF90EF900895DD
:1007A000AF92BF92CF92DF92FF920F931F93CF939E
:1007B000DF936C018B01F42E590162E040E00E944E
:1007C0006003C6016AE044E00E946003C60164E180
:1007D00040E80E94BC03C60162E14F2D98010E94CF
:1007E0003003C60162E043E00E946003C8E8D3E141
:1007F000C6016AE00E94120382FD04C02197C1F77E
:1008000084E012C0C60162E040E00E946003C601BD
:1008100064E40E941203F5018083C60162E40E9431
:100820001203F501818381E0DF91CF911F910F9138
:10083000FF90DF90CF90BF90AF9008952F923F929E
:100840004F925F926F927F928F929F92AF92BF92E0
:10085000CF92DF92EF92FF920F931F93DF93CF938C
:1008600000D00F92CDB7DEB73C01962E4B83190115
:1008700027017601A114B10411F410E002C0F501C2
:100880001081C30162E040E00E946003C30168E0A0
:100890004FE70E946003C30164E140E80E94BC038B
:1008A000C30162E1402F91010E943003882D82959F
:1008B000807F180FC3016AE1412F0E946003C301CA
:1008C00062E0492D0E946003FCE09F1629F4C301F9
:1008D0006AE140E80E94BC0300ED17E08B81C82E5E
:1008E000DD24C30168E00E941203282F30E0C90113
:1008F0008C219D21892B31F420FD6AC001501040CC
:1009000081F766C0C3016CE00E941203C82EDD248B
:10091000C60183719070009711F042E05EC04114EF
:10092000510409F1E114F104F1F0C30164E10E9402
:100930001203482FF7018081841710F445E04DC061
:10094000F7014083C30162E19201082D0E94B302C6
:10095000C30168E10E941203982F9770A114B1049B
:1009600011F0F5019083C3FE02C043E036C041148C
:10097000510491F1E114F10479F1888D882361F13A
:10098000F7014081413021F4943021F549E025C040
:10099000423000F19923F1F44250C301B2019E01AB
:1009A0002F5F3F4F0E94D003482F8130B1F4F701F1
:1009B0008081F201E80FF11D329790813296898192
:1009C000981741F4319790818A81981719F405C0DE
:1009D00044E003C048E001C041E0842F0F900F9035
:1009E0000F90CF91DF911F910F91FF90EF90DF90CB
:1009F000CF90BF90AF909F908F907F906F905F90BF
:100A00004F903F902F9008954F925F926F927F92F8
:100A10008F92AF92BF92CF92DF92EF92FF920F939D
:100A20001F93CF93DF93FB01542FD9013801270186
:100A30008C2C0F92CDB7DEB7A9826CE040E39F010A
:100A4000052F7D01630152010E941E040F90DF916A
:100A5000CF911F910F91FF90EF90DF90CF90BF90BB
:100A6000AF908F907F906F905F904F9008958F928E
:100A70009F92AF92CF92EF92FF920F931F93DF93CB
:100A8000CF9300D0CDB7DEB78C016A837A014901DC
:100A90004115510529F1F9018081823008F1C80121
:100AA0006CE140E80E94A70387E08983C801BE018A
:100AB0006E5F7F4F41E0970184017E010894E11C45
:100AC000F11CCC24AA240E940405982F813059F4EB
:100AD000F4018081823031F48981882321F002C0C1
:100AE00095E001C092E0892F0F900F90CF91DF9198
:100AF0001F910F91FF90EF90CF90AF909F908F90AC
:100B00000895FB019A0166E2AF010E94370508953E
:100B1000DF93CF9300D00F92CDB7DEB722E02983C9
:100B2000BE016E5F7F4FAE014F5F5F4F0E94810538
:100B3000982F813019F080E0933009F481E00F9014
:100B40000F900F90CF91DF9108952F923F924F9287
:100B50005F926F927F928F929F92AF92BF92CF924D
:100B6000DF92EF92FF920F931F93DF93CF93CDB756
:100B7000DEB72C970FB6F894DEBF0FBECDBF2C01A9
:100B80001B014C87413510F017E05CC16CE140E877
:100B90000E94A703BB24B39482E0B81691F0E3E06F
:100BA000BE16D9F0F1E0BF1609F047C183E98B8387
:100BB0008C858823B1F0F1018081853090F080E050
:100BC0000AC0F5E9FB838C85882369F0F1018081F7
:100BD000883048F083E041E008C087E98B8386E0F5
:100BE00003C080E001C083E040E0682E7724C301A9
:100BF000B3E0880F991FBA95E1F7DC84D81AD7FCC7
:100C0000DD24442311F452E003C088E88D8353E0CF
:100C100090E08D2D877009F091E08D2D859585955B
:100C20008595890F09F1442311F494E001C093E004
:100C3000891708F4982F0894611C711CD101A60D26
:100C4000B71D08946108710820E030E0852F820FFD
:100C5000E3E0F0E0EC0FFD1FE80FF11D8D918083C4
:100C60002F5F3F4F291790F3442311F0F8E0DF0E78
:100C70008FE18D1514F5E0E7EC8328858F81282717
:100C80008E819D81892728272987C201BE016D5F3A
:100C90007F4F47E09E01265F3F4F0E94D003182FF1
:100CA000813009F0CFC01982F3E0FA8319E0A9E09E
:100CB0008A2E912C8C0E9D1E21C08D2D68E00E94E5
:100CC000560D99838D2DD7FC895F282F2595259565
:100CD00025952E5F822F8295807F890F8C8340E03F
:100CE000911141E0142F120FF3E08F2E912C8C0EF6
:100CF0009D1E820E911C89E0821B8A83C9804C2D27
:100D00004295407F4C0DC2016AE10E946003C2011E
:100D1000BE016D5F7F4F412F94018E010E5F1F4F0B
:100D20007E010894E11CF11CAA240E940405182FDE
:100D30008330B9F5C2016CE10E94120385FD82C0C7
:100D4000482F4F7109F440E2242F30E08D2D992770
:100D500087FD9095821793070CF06FC0D42E842FD7
:100D6000992787FD9095019787709070982F242F71
:100D70002595259525952F5F30E0811131E0230FD2
:100D8000E3E0F0E0EC0FFD1FE20FF11D21E030E0A9
:100D900002C0220F331F9A95E2F78081822B808355
:100DA00067CF813009F04EC08FE18D151CF0E0E275
:100DB000DE2E61CF8D81883819F044E092E002C0C8
:100DC00043E093E0D3011196A20DB31D20E030E083
:100DD000892F820FE3E0F0E0EC0FFD1FE80FF11D1B
:100DE00080818D932F5F3F4F241790F30A8103304A
:100DF00031F58981882319F5C201B40141E09E01D2
:100E00002B5F3F4F0E94D003182F8130D9F49D8172
:100E1000F40181819817A9F49E818281981789F441
:100E2000208122FF02C0B394B7CEF1012387B09E88
:100E3000C00111248F5F808305C016E003C012E05B
:100E400001C018E0812F2C960FB6F894DEBF0FBEBC
:100E5000CDBFCF91DF911F910F91FF90EF90DF9069
:100E6000CF90BF90AF909F908F907F906F905F904A
:100E70004F903F902F900895BC0140E00E94A5053F
:100E800090E0813009F491E0892F0895CF93DF93AA
:100E9000EC018D850E949F09892B59F48D8561E0B5
:100EA0000E944B0962E370E080E090E00E946E08CF
:100EB00003C0CE010E949103CE0164E540E80E9488
:100EC0006003CE0166E549EA0E946003CE0168E551
:100ED00043E00E946003CE016AE548EE0E94600391
:100EE000CE016AE240E40E946003CE0162E24DE37B
:100EF0000E946003CE010E947F03DF91CF9108958D
:100F000081E00E948E0280E00E9497020895FF9285
:100F10000F931F938C01862FF42EF801648761E0F4
:100F20000E940C09F801848561E00E944B09F801D8
:100F3000F5868F2D61E00E940C09F801858560E03F
:100F40000E944B09C8010E9480071F910F91FF90DA
:100F50000895823000F5E82FF0E0EE0FFF1FE85112
:100F6000FE4F71836083882319F08130A1F408C09B
:100F7000809169008C7F842B80936900E89A0895A2
:100F800080916900440F551F440F551F837F842BA8
:100F900080936900E99A08951F920F920FB60F92FD
:100FA00011242F933F934F935F936F937F938F936E
:100FB0009F93AF93BF93EF93FF938091E80190913C
:100FC000E901892B29F0E091E801F091E901099507
:100FD000FF91EF91BF91AF919F918F917F916F9111
:100FE0005F914F913F912F910F900FBE0F901F90E7
:100FF00018951F920F920FB60F9211242F933F93C3
:101000004F935F936F937F938F939F93AF93BF9310
:10101000EF93FF938091EA019091EB01892B29F0E6
:10102000E091EA01F091EB010995FF91EF91BF91F9
:10103000AF919F918F917F916F915F914F913F9170
:101040002F910F900FBE0F901F9018951F920F9227
:101050000FB60F9211242F933F938F939F93AF93CB
:10106000BF938091F0019091F101A091F201B091B4
:10107000F3013091F4010196A11DB11D232F2D5FC5
:101080002D3720F02D570196A11DB11D2093F4019D
:101090008093F0019093F101A093F201B093F301DA
:1010A0008091EC019091ED01A091EE01B091EF01E2
:1010B0000196A11DB11D8093EC019093ED01A093C9
:1010C000EE01B093EF01BF91AF919F918F913F914E
:1010D0002F910F900FBE0F901F9018959B01AC01A0
:1010E0007FB7F8948091EC019091ED01A091EE0111
:1010F000B091EF0166B5A89B05C06F3F19F001964E
:10110000A11DB11D7FBFBA2FA92F982F8827860F49
:10111000911DA11DB11D62E0880F991FAA1FBB1F61
:101120006A95D1F7BC012DC0FFB7F8948091EC010E
:101130009091ED01A091EE01B091EF01E6B5A89B71
:1011400005C0EF3F19F00196A11DB11DFFBFBA2FD9
:10115000A92F982F88278E0F911DA11DB11DE2E0A8
:10116000880F991FAA1FBB1FEA95D1F7861B970B03
:10117000885E9340C8F22150304040405040685152
:101180007C4F211531054105510571F608950197F0
:1011900039F0880F991F880F991F02970197F1F76F
:1011A0000895789484B5826084BD84B5816084BDDF
:1011B00085B5826085BD85B5816085BDEEE6F0E0D0
:1011C000808181608083E1E8F0E01082808182602C
:1011D0008083808181608083E0E8F0E080818160AD
:1011E0008083E1EBF0E0808184608083E0EBF0E0DD
:1011F000808181608083EAE7F0E080818460808381
:10120000808182608083808181608083808180682A
:1012100080831092C1000895CF93DF93482F50E050
:10122000CA0186569F4FFC0134914A575F4FFA011D
:101230008491882369F190E0880F991FFC01E85997
:10124000FF4FA591B491FC01EE58FF4FC591D49189
:10125000662351F42FB7F8948C91932F909589239E
:101260008C93888189230BC0623061F42FB7F89486
:101270008C91932F909589238C938881832B8883DD
:101280002FBF06C09FB7F8948C91832B8C939FBF80
:10129000DF91CF910895482F50E0CA0182559F4FAA
:1012A000FC012491CA0186569F4FFC0194914A5734
:1012B0005F4FFA013491332309F440C0222351F1E6
:1012C000233071F0243028F42130A1F0223011F5C0
:1012D00014C02630B1F02730C1F02430D9F404C056
:1012E000809180008F7703C0809180008F7D8093F4
:1012F000800010C084B58F7702C084B58F7D84BD17
:1013000009C08091B0008F7703C08091B0008F7DBD
:101310008093B000E32FF0E0EE0FFF1FEE58FF4F79
:10132000A591B4912FB7F894662321F48C919095F0
:10133000892302C08C91892B8C932FBF0895682F2D
:1013400070E0CB0182559F4FFC012491CB01865662
:101350009F4FFC0144916A577F4FFB019491992361
:1013600019F420E030E03CC0222351F1233071F029
:10137000243028F42130A1F0223011F514C0263099
:10138000B1F02730C1F02430D9F404C0809180003E
:101390008F7703C0809180008F7D8093800010C084
:1013A00084B58F7702C084B58F7D84BD09C08091DC
:1013B000B0008F7703C08091B0008F7D8093B00024
:1013C000892F90E0880F991F84589F4FFC01A591A9
:1013D000B4918C9120E030E0842311F021E030E0E2
:1013E000C901089508951F920F920FB60F9211240C
:1013F0002F933F934F938F939F93EF93FF938091FE
:10140000C00082FD1DC04091C60020913502309180
:1014100036022F5F3F4F2F733070809137029091CB
:1014200038022817390771F0E0913502F091360241
:10143000EB50FE4F4083309336022093350202C0BA
:101440008091C600FF91EF919F918F914F913F91B5
:101450002F910F900FBE0F901F901895E091890269
:10146000F0918A02E05CFF4F81919191208131815E
:10147000805C9F4F821B930B60E470E00E94630DC1
:10148000892B11F00E94F20908951F920F920FB656
:101490000F9211242F933F938F939F93EF93FF937A
:1014A0002091790230917A0280917B0290917C02A6
:1014B0002817390731F48091C1008F7D8093C100D6
:1014C00014C0E0917B02F0917C02E75CFD4F20812B
:1014D00080917B0290917C0201968F739070909323
:1014E0007C0280937B022093C600FF91EF919F9135
:1014F0008F913F912F910F900FBE0F901F901895D5
:10150000AF92BF92DF92EF92FF920F931F93CF9310
:10151000DF93EC017A018B01DD24403081EE580726
:1015200080E0680780E0780711F0DD24D39491E033
:10153000A92EB12CEC89FD89DD2069F0C50108A038
:1015400002C0880F991F0A94E2F7808360E079E077
:101550008DE390E005C0108260E874E88EE190E0D1
:10156000A80197010E94760D215030404040504024
:10157000569547953795279580E12030380720F01C
:10158000DD2011F0DD24D6CFE889F9893083EA899E
:10159000FB89208319A2EE89FF89408121E030E098
:1015A000C9010C8C02C0880F991F0A94E2F7482BDE
:1015B0004083EE89FF894081C9010D8C02C0880FEC
:1015C000991F0A94E2F7482B4083EE89FF894081F6
:1015D000C9010E8C02C0880F991F0A94E2F7482BAC
:1015E0004083EE89FF8980810F8C02C0220F331F58
:1015F0000A94E2F7209528232083DF91CF911F9151
:101600000F91FF90EF90DF90BF90AF900895DC01B5
:101610001C96ED91FC911D97E05CFF4F819191919B
:1016200020813181805C9F4F821B930B60E470E0CE
:101630000E94630D0895DC011C96ED91FC911D97AD
:10164000E05CFF4F20813181E054F040DF01AE5B70
:10165000BF4F8D919C9111972817390719F42FEFDF
:101660003FEF07C08D919C91E80FF91F8081282FD3
:1016700030E0C9010895DC011C96ED91FC911D97A5
:10168000E05CFF4F20813181E054F040DF01AE5B30
:10169000BF4F8D919C9111972817390719F42FEF9F
:1016A0003FEF10C08D919C911197E80FF91F208199
:1016B0008D919C91119701968F73907011969C93C8
:1016C0008E9330E0C9010895DC0191968C91919739
:1016D000882339F05496ED91FC915597808186FFCF
:1016E000F9CF91961C920895CF93DF93EC01EE858C
:1016F000FF85E05CFF4F20813181E054F0402F5F97
:101700003F4F2F733070DF01AE5BBF4F8D919C91C7
:10171000119728173907D1F3E05CFF4F8081918141
:10172000E054F040E80FF91F6083EE85FF85E05C30
:10173000FF4F31832083EE89FF89208181E090E093
:101740000F8C02C0880F991F0A94E2F7282B208380
:1017500081E089A3EC89FD8980818064808381E0B8
:1017600090E0DF91CF91089581E00895109280027A
:1017700010927F0288EE93E0A0E0B0E080938102B7
:1017800090938202A0938302B09384028BEB91E04A
:1017900090937E0280937D0285EF91E090938A0280
:1017A0008093890289E392E090938C0280938B026C
:1017B00085EC90E090938E0280938D0284EC90E013
:1017C0009093900280938F0280EC90E0909392022D
:1017D0008093910281EC90E0909394028093930225
:1017E00082EC90E0909396028093950286EC90E0D4
:1017F000909398028093970284E08093990283E00B
:1018000080939A0287E080939B0285E080939C02FC
:1018100081E080939D0208950895CF93DF930E9405
:10182000D1080E940C0C0E942D02CEE2DAE00E9448
:1018300060012097E1F30E942E0AF9CFCF92DF9248
:10184000EF92FF920F931F93CF93DF937C016B0175
:101850008A01C0E0D0E00FC0D6016D916D01D701C3
:10186000ED91FC910190F081E02DC7010995C80F21
:10187000D91F015010400115110571F7CE01DF91FC
:10188000CF911F910F91FF90EF90DF90CF9008952F
:10189000EF92FF920F931F938C01DC01ED91FC916D
:1018A0000190F081E02D6DE009957C01D801ED916A
:1018B000FC910190F081E02DC8016AE009959C013E
:1018C0002E0D3F1DC9011F910F91FF90EF900895BC
:1018D000CF93DF93EC016115710519F420E030E03E
:1018E0000FC0DB010D900020E9F71197A61BB70B85
:1018F000E881F9810280F381E02DAD0109959C0119
:10190000C901DF91CF9108954F925F927F928F929C
:101910009F92AF92BF92CF92DF92EF92FF920F937E
:101920001F93DF93CF93CDB7DEB7A1970FB6F8948F
:10193000DEBF0FBECDBF2C01742ECB01223008F4C8
:101940002AE019A231E2C32ED12CCC0EDD1E822E4C
:101950009924AA24BB24672D752FA50194010E9408
:10196000760D79018A01C801B701A50194010E9491
:10197000370D472D461B0894C108D1084A3014F48E
:10198000405D01C0495CF6014083E114F1040105AA
:10199000110521F07E2C5F2DC801DDCFC201B601FB
:1019A0000E94680CA1960FB6F894DEBF0FBECDBFA3
:1019B000CF91DF911F910F91FF90EF90DF90CF902B
:1019C000BF90AF909F908F907F905F904F900895C1
:1019D000DC012115310541F4ED91FC910190F0817C
:1019E000E02D642F099508950E94840C0895EF92CC
:1019F000FF920F931F939A017B0100E010E0B80162
:101A0000A7010E94E80C1F910F91FF90EF9008959D
:101A1000EF92FF920F931F939A01E62EFF2400E0AE
:101A200010E0B801A7010E94E80C1F910F91FF90F0
:101A3000EF9008950E94680C0895EF92FF920F9323
:101A40001F937C010E94680C8C01C7010E94480C06
:101A5000080F191FC8011F910F91FF90EF90089573
:101A600070E0382F20E0622B732BCB010895629F2A
:101A7000D001739FF001829FE00DF11D649FE00D86
:101A8000F11D929FF00D839FF00D749FF00D659FE7
:101A9000F00D9927729FB00DE11DF91F639FB00DE6
:101AA000E11DF91FBD01CF011124089587FB082E08
:101AB000062687FD819567FD61953AD00EF49195D4
:101AC00007FC8195089597FB092E07260AD077FD1C
:101AD00004D03AD006D000201AF4709561957F4F5B
:101AE0000895F6F7909581959F4F0895A1E21A2EDB
:101AF000AA1BBB1BFD010DC0AA1FBB1FEE1FFF1FB2
:101B0000A217B307E407F50720F0A21BB30BE40B01
:101B1000F50B661F771F881F991F1A9469F7609548
:101B20007095809590959B01AC01BD01CF01089502
:101B3000991B79E004C0991F961708F0961B881F1F
:101B40007A95C9F780950895AA1BBB1B51E107C080
:101B5000AA1FBB1FA617B70710F0A61BB70B881F3D
:101B6000991F5A95A9F780959095BC01CD010895CC
:101B7000EE0FFF1F0590F491E02D0994F894FFCF2C
:101B80005549442053697A653A20004361726420C4
:101B900055494428686578293A00200020300043E0
:101BA000617264205549442862696E293A00507375
:101BB0006575646F49442862696E293A20000052B5
:101BC0004649442D5338382D6C696768742D30327E
:101BD000783136763038004D465243353232205314
:101BE0006F6674776172652056657273696F6E3ABD
:101BF000203078005741524E494E473A20436F6D8E
:101C00006D756E69636174696F6E206661696C756C
:101C100072652C20697320746865204D46524335E7
:101C200032322070726F7065726C7920636F6E6EE5
:101C300065637465643F0000000000740B1E0C07B0
:081C40000B3B0B1B0B640B00B6
:00000001FF
